:100000000C94A3020C94DB020C94DB020C94DB0234
:100010000C94DB020C94DB020C94DB020C94DB02EC
:100020000C94DB020C94DB020C940A250C94DC2566
:100030000C94FE1F0C94DB020C94DB020C94DB028C
:100040000C94DB020C94DB020C94DB020C94DB02BC
:100050000C94DB020C9486200C94DB020C94DB02E3
:100060000C94DB020C94DB020C94DB020C94DB029C
:100070000C94DB020C94DB020C94DB020C94DB028C
:100080000C94DB020C94DB020C94DB020C94DB027C
:100090000C94DB020C94DB020C94DB020C94DB026C
:1000A0000C94DB020C94DB020C94DB020E050E05B3
:1000B0003A053A05A205C005D806D806CB05640660
:1000C0007506750649267026682770266827BC269F
:1000D000DF26682736274527165C14001A0008001B
:1000E000150017001C0018000C00120013002A0055
:1000F0002B4204001600070009000A000B000D0047
:100100000E000F0033002800E1001D001B00060058
:1001100019000500050011001000360037005200DC
:10012000E000E2000000E3002C4100002C002C4124
:10013000500051004F000251005C1E001F002000C3
:1001400021002200230024002500260027000000B3
:1001500049003A003B003C003D003E003F002D00BE
:100160002E002F003000310000004000410042000E
:1001700043004400450000000000000000000000B3
:10018000AA00A8000000A900010000000100000072
:100190000000000000000000005C00000000000003
:1001A000000000000000000000000000000000004F
:1001B000000000000000000000000000000000003F
:1001C000000000000000000000000000000000002F
:1001D000000000000000000000000000000000001F
:1001E000000000000000000000000000000000000F
:1001F000000000000000000000047F3F1F64321474
:10020000643214783C1E1E140A0522232526282950
:100210002A2C2D2F3032333536383A3B3D3E404282
:10022000434547494A4C4E5051535557595A5C5EC5
:100230006062646668696B6D6F71737577797B7DD9
:100240007F81838587898A8C8E90929496989A9CD8
:100250009E9FA1A3A5A7A8AAACAEAFB1B3B4B6B8F0
:10026000B9BBBCBEBFC1C2C3C5C6C7C9CACBCCCD52
:10027000CED0D1D2D2D3D4D5D6D7D7D8D9D9DADA2D
:10028000DBDBDBDCDCDCDCDCDDDDDDDDDCDCDCDCAD
:10029000DCDBDBDBDADAD9D9D8D7D7D6D5D4D3D2E1
:1002A000D2D1D0CECDCCCBCAC9C7C6C5C3C2C1BFBF
:1002B000BEBCBBB9B8B6B4B3B1AFAEACAAA8A7A523
:1002C000A3A19F9E9C9A98969492908E8C8A8987DF
:1002D0008583817F7D7B79777573716F6D6B6968BD
:1002E000666462605E5C5A5957555351504E4C4A91
:1002F0004947454342403E3D3B3A3836353332303C
:100300002F2D2C2A292826252322FFAA7F5540009D
:1003100001010101010101010102020202020202C6
:100320000202030303030303030304040404040499
:10033000040505050505060606060607070707075F
:1003400008080808090909090A0A0A0B0B0B0C0C12
:100350000C0D0D0D0E0E0E0F0F0F101011111112AE
:100360001213131414151516161717181819191A2D
:100370001A1B1B1C1D1D1E1E1F2020212222232490
:1003800024252626272829292A2B2C2D2D2E2F30CF
:10039000313232333435363738393A3B3C3D3E3FE3
:1003A000404142434445464748494A4C4D4E4F50D0
:1003B000515354555658595A5B5D5E5F616264658E
:1003C0006668696B6C6D6F7072737577787A7B7D18
:1003D0007E8082838587888A8C8E8F91939596986C
:1003E0009A9C9EA0A2A3A5A7A9ABADAFB1B3B5B788
:1003F000BABCBEC0C2C4C6C9CBCDCFD1D4D6D8DB5F
:10040000DDDFE2E4E7E9EBEEF0F3F5F8FAFDFF0AF1
:100410000342006F006C00740000001C034C00419C
:10042000005A005900440045005300490047004E5F
:100430000045005200530000000403090409023B78
:1004400000020100A0FA09040000010301010009F3
:100450002111010001224000070581030800010964
:100460000401000103000000092111010001227BA9
:1004700000070582032000011201000200000008AD
:10048000444C410001000102000105010902A101E3
:1004900085020901A1000509190129081500250196
:1004A0009508750181020501093009311581257F03
:1004B00095027508810609381581257F9501750813
:1004C0008106050C0A38021581257F950175088182
:1004D00006C0C005010980A101850319012AB700E2
:1004E000150126B700950175108100C0050C0901A2
:1004F000A101850419012AA002150126A002950177
:1005000075108100C005010906A101050719E02940
:10051000E71500250195087501810295017508818F
:10052000010507190029FF150026FF00950675082B
:1005300081000508190129059505750191029501AC
:1005400075039101C00011241FBECFEFDAE0DEBFBA
:10055000CDBF04B603FE18C08091D1029091D202A3
:10056000A091D302B091D4028730904BA740B04BFA
:1005700059F41092D1021092D2021092D30210922A
:10058000D402E0E0F8E3099511E0A0E0B1E0E6E391
:10059000F1E502C005900D92A43CB107D9F722E025
:1005A000A4ECB1E001C01D92A13DB207E1F70E94A9
:1005B000E7120C9499280C94000081E0089581E0E2
:1005C00008950C94DF0208950C94E3021F93CF93D7
:1005D000DF9300D000D01F92CDB7DEB749835A8396
:1005E0006B833091C70189819A81311114C06623D0
:1005F00059F0222349F00E941509182F682F89818C
:100600009A810E94BE0803C00E94E908182F6981E0
:100610007A81812F04C00E94150969817A810F9027
:100620000F900F900F900F90DF91CF911F910C942E
:100630004F10FC01262F408151816281738184819A
:100640000C94E60281E00895CF93DF93EC0160E023
:100650000E941903BE01DF91CF910C94E4020C9427
:1006600098110C94941108950E9468070E94330316
:100670002FEF84E39CE0215080409040E1F700C0E0
:1006800000000C94AC200F931F93CF93DF938C0149
:1006900061E00E941903EC01B8010E94E102882385
:1006A00009F444C0B801CE010E94C91E8823F1F1AB
:1006B000B801CE010E94DD1C8823C1F1B801CE0132
:1006C0000E94251E882391F1B801CE010E94E31BF0
:1006D000882361F1F8018281882309F1CB358DE50A
:1006E000D807C1F050F4C115FCE5DF0781F0CF3D1C
:1006F000DC45A9F40E944C0E19C0CC35EDE5DE07AF
:1007000061F0CD35DD4559F40E948F0D08C00E947F
:1007100034030CC00E94980D02C00E949B0DC801BA
:10072000DF91CF911F910F910C94DD0280E0DF915A
:10073000CF911F910F9108950E94E01F0E94B9036D
:100740000C94601A0E94BC030E942C1B0C94E61FA0
:1007500008950C94A80381E008950C94AB030895C8
:10076000CF93C82F0E94A9038C2F0E94AD03CF9175
:10077000089580E00C94B0030E94251F0C94B003F0
:100780000E94251F9091C601891721F08093C60110
:100790000C94B0030895CF93DF93CDB7DEB72B97BA
:1007A0000FB6F894DEBF0FBECDBF4F835887698761
:1007B0007A878B8761110E94DB0C9E012F5F3F4F70
:1007C00086E0F90111928A95E9F785E0FE013796F6
:1007D000D90101900D928A95E1F789819A814C8126
:1007E0005D81452B31F09F3F31F491E08F3F19F44B
:1007F00003C091E001C090E090FF09C049815A8197
:100800006B817C818D819E810E94FC0B05C0C9019A
:100810000E9422038111F2CF2B960FB6F894DEBF0F
:100820000FBECDBFDF91CF910895FC0180819181F2
:100830000E9457090895CF93882309F450C0C82F08
:100840008CEF8C0F813AD0F46C2F80910201909143
:1008500003010E94821F882349F06C2F80910201BE
:10086000909103010E94BA1F0E94FD0C6C2F809191
:100870000201909103010E94B81F0CC080E28C0F0E
:10088000883058F4C77081E001C0880FCA95EAF734
:100890000E94BE0CCF910C94FD0CEBE5EC0FE33005
:1008A00040F4F0E0E65AFE4F808190E0CF910C9446
:1008B0004A1FE8E5EC0FE73150F4F0E0EE0FFF1FC0
:1008C000E45DFE4F80819181CF910C94601FCD3EFD
:1008D00030F08C2F0E946C13CF910C943E14CF916A
:1008E0000895882389F19CEF980F913A40F4682F7E
:1008F00080910201909103010E94BA1F0DC090E205
:10090000980F983058F4877091E001C0990F8A953C
:10091000EAF7892F0E94C40C0C94FD0C9BE5980FFC
:10092000933020F480E090E00C944A1F98E5980FF3
:10093000973120F480E090E00C94601F8D3E20F011
:100940000E94C7130C943E1408951F93CF93DF9316
:10095000182FEB010E941B04209741F08FE99FE0C4
:100960000197F1F700C000002197F6CF812FDF91AA
:10097000CF911F910C947104893319F060E070E0FD
:1009800002C060E570E00C94A504882321F00E9469
:10099000BE0C0C94FD0C0895882321F00E94C40C19
:1009A0000C94FD0C0895CF92DF92EF92FF920F937B
:1009B0001F93CF93DF937C01D62FC72FFC011281A9
:1009C000058102950F700E94B40C8823B9F01123A1
:1009D000A9F08C2F807F803421F080E28D0F883049
:1009E00068F08091830282FD09C082E00E945D0D63
:1009F0000E94B40C91E0D82ED92601C0D12CCC2E67
:100A0000C2948FE0C8228C2D90E08C30910508F0C4
:100A1000CFC1FC01EA5AFF4F0C94F4278C2F807F42
:100A2000CF70882311F0C295C07F112399F0CC2399
:100A300009F4AAC180E28D0F883010F0D11104C0F2
:100A40008C2F0E94BE0C03C08C2F0E94CE0C0E94E3
:100A5000FD0C9AC18D2F0E947104CC2309F4A8C10A
:100A600080E28D0F883038F1DD2329F18C2F0E9430
:100A7000D40C24C08C2F807FCF70803211F0C295AF
:100A8000C07FDD2319F0D130A1F13DC080918302F8
:100A900082FF17C0112349F0CC2329F08C2F0E942C
:100AA000BE0C0E94FD0C80E070C180E00E947104C9
:100AB000CC2309F47DC18C2F0E94C40C0E94FD0C34
:100AC00077C1112371F0002341F0013031F40E940D
:100AD000DE0C8C2B0E94E60C6BC10E94DE0C8C2B72
:100AE0001DC0002319F0013009F462C10E94F30C0B
:100AF00025C0112321F0063008F05AC10EC0053080
:100B000008F056C11BC0112361F0002331F0F7013A
:100B1000858180FF39C18F7085838C2F0E94C50429
:100B200047C1002359F0D93309F03FC1FFEF07EE69
:100B300013E0F15000401040E1F735C18C2F0E94C6
:100B4000CC0436C18C2F86958695837019F0813040
:100B500061F02EC1112321F08D2F9C2F937002C0C4
:100B600080E090E00E944A1F2BC1112321F08D2FBD
:100B70009C2F937002C080E090E00E94601F20C113
:100B80008D2F112319F00E946C1302C00E94C7130D
:100B90000E943E1415C18C2F837009F047C01111BB
:100BA0000BC12D2F229526952770220F220F6D2F16
:100BB0006F70862F90E0A0E0B0E0022E04C0880F96
:100BC000991FAA1FBB1F0A94D2F7D4FF10C04FE091
:100BD00050E060E070E004C0440F551F661F771FAF
:100BE0002A95D2F7409550956095709503C040E0E6
:100BF00050E0BA01C695C695C3708A019B01082BC7
:100C0000192B2A2B3B2BC901B801C23049F058F4EB
:100C1000C13019F00E94D407CFC00E94C207CCC0D7
:100C20000E94E607C9C00E94C007C6C0112319F080
:100C30008C2F817001C08695882309F4BDC02D2FAB
:100C4000229526952770220F220F6D2F6F70862F09
:100C500090E0A0E0B0E0022E04C0880F991FAA1F08
:100C6000BB1F0A94D2F7D4FF10C04FE050E060E001
:100C700070E004C0440F551F661F771F2A95D2F7F6
:100C8000409550956095709503C040E050E0BA01E2
:100C9000C695C695C3708A019B01082B192B2A2B78
:100CA0003B2BC901B801C23049F058F4C13019F0EA
:100CB0000E94990881C00E9487087EC00E94AB08EC
:100CC0007BC00E94FA0778C0CF70112339F08C2FB7
:100CD0000E9420088D2F0E94C5046EC08D2F0E9497
:100CE000CC048C2F0E94410867C0D23F21F128F428
:100CF000D03F41F0D13FC1F043C0D33F19F1D43FC1
:100D000079F03EC0112341F0053008F051C08C2F1E
:100D10008F710E9466084CC0063008F049C0F7CFBA
:100D20008091830282FF18C0112339F08C2F8F71BC
:100D30000E9420083DC01123C9F38C2F8F710E949F
:100D4000410836C0112329F08C2F8F710E940B08A7
:100D50002FC00E9406082CC0112349F0CF718C2FA0
:100D60000E94200863E08C2F0E94420D21C081E088
:100D70000E945D0D0230E0F082E00E945D0D18C01F
:100D8000112331F0002391F28D2F0E941B0410C01B
:100D9000002399F2D93349F41FEF27EE33E01150C5
:100DA00020403040E1F700C000008D2F0E94710408
:100DB00088EF8C0D843020F40E94251F0E94B00320
:100DC000DD20C9F00E94B00C80FD15C0F701128231
:100DD0000E94AA0C0E942008C7010E941C070E94C2
:100DE000AA0CDF91CF911F910F91FF90EF90DF90B0
:100DF000CF900C944108DF91CF911F910F91FF90FC
:100E0000EF90DF90CF9008950F931F93CF93DF93D0
:100E1000EC01688179818A810E9462098C010E94BB
:100E2000BD080E94AE07B801CE010E94D304DF9135
:100E3000CF911F910F910895CF93DF93EC0198818B
:100E400089812B813C81232B31F08F3F31F481E06C
:100E50009F3F19F403C081E001C080E080FD1DC008
:100E6000CE010E944303811110C00E94B40C88235C
:100E7000A1F08A81882389F08091830282FD0DC0D0
:100E800082E0DF91CF910C945D0DCE010E940407AA
:100E9000CE01DF91CF910C942403DF91CF9108957F
:100EA00080E090E00E944A1F80E090E00E94601F76
:100EB0000E94DB0C0E94FD0C0E946F150C943E14E6
:100EC00080910201909103010E94BC1F0C94500775
:100ED0000E94CB0C0C94600792959F70963079F02D
:100EE00010F4925001C09A50923068F4803F69F03B
:100EF00018F4883E40F409C0843F29F406C0883EB7
:100F000020F0813F11F080E0089581E00895FC0118
:100F1000808191810E9457090E946C070895CF93A8
:100F2000DF9300D000D01F92CDB7DEB70F900F90A7
:100F30000F900F900F90DF91CF910895CF93DF9393
:100F400000D000D000D0CDB7DEB726960FB6F8940B
:100F5000DEBF0FBECDBFDF91CF91089508950895F4
:100F60000C94AF070C94B0070E94B2076093EA019B
:100F70007093EB018093EC019093ED010C9450077A
:100F80000C94B4070F931F930091EA011091EB01A9
:100F90002091EC013091ED01602B712B822B932B72
:100FA0001F910F910C94B4070F931F930091EA01C6
:100FB0001091EB012091EC013091ED016023712340
:100FC000822393231F910F910C94B4070F931F93C7
:100FD0000091EA011091EB012091EC013091ED01BB
:100FE00060277127822793271F910F910C94B407D4
:100FF0000C94AF070E94F8076093E6017093E70135
:101000008093E8019093E9010C94500760E070E050
:10101000CB010C94FA070F931F9341E050E060E07E
:1010200070E08A019B0104C0000F111F221F331FB3
:101030008A95D2F7C901B8011F910F910C94FA0754
:101040000F931F9341E050E060E070E004C0440F54
:10105000551F661F771F8A95D2F78091E601909100
:10106000E701A091E801B091E9018A019B01082BF9
:10107000192B2A2B3B2BC901B8011F910F910C94FE
:10108000FA070F931F9341E050E060E070E004C066
:10109000440F551F661F771F8A95D2F740955095CC
:1010A000609570958091E6019091E701A091E8012B
:1010B000B091E9018A019B01082319232A233B23CC
:1010C000C901B8011F910F910C94FA070F931F9358
:1010D00041E050E060E070E004C0440F551F661F1F
:1010E000771F8A95D2F78091E6019091E701A09150
:1010F000E801B091E9018A019B01082719272A27F5
:101100003B27C901B8011F910F910C94FA070F9367
:101110001F930091E6011091E7012091E8013091C1
:10112000E901602B712B822B932B1F910F910C9453
:10113000FA070F931F930091E6011091E7012091A8
:10114000E8013091E90160237123822393231F91E9
:101150000F910C94FA070F931F930091E6011091E1
:10116000E7012091E8013091E9016027712782278A
:1011700093271F910F910C94FA0708952CE0929FEA
:10118000800D1124E82FE695E695E695877051E0ED
:1011900001C0550F8A95EAF785E0E89FF001112418
:1011A000E853FE4F20E030E070E04081CB01022E9A
:1011B00002C0969587950A94E2F7817081958427FD
:1011C0008523842781932F5F3F4F2530310569F7B1
:1011D00008952CE0929F800D1124682F66956695E6
:1011E0006695982F977085E0689FB001112440E0C4
:1011F00050E080E0FB01E40FF51FE853FE4F208133
:1012000030E0092E02C0369527950A94E2F7217046
:101210003327042E01C0220F0A94EAF7822B4F5F76
:101220005F4F4530510531F70895BF92CF92DF925D
:10123000EF92FF920F931F93CF93DF938C01C09097
:10124000E601D090E701E090E801F090E90180919B
:10125000EA019091EB01A091EC01B091ED01C82A57
:10126000D92AEA2AFB2ACFE1D0E0D701C6010C2E09
:1012700004C0B695A795979587950A94D2F780FDF7
:1012800004C0219790F7B12C07C0BC2EB8018C2F59
:101290000E9462100197A9F38B2DDF91CF911F91CE
:1012A0000F91FF90EF90DF90CF90BF900895CF9374
:1012B000DF93EC010E941509BE010E946210DF91CC
:1012C000CF9108951F93CF93DF93EB019091C701C6
:1012D000992321F0CB010E94570913C0882349F0BC
:1012E000CB010E941509182F682FCE010E94BE085D
:1012F00004C0CB010E94E908182FBE01812F0E9473
:101300006210DF91CF911F9108951F93CF93DF93C8
:10131000C091EE0116E08091EF01C81799F0D0E07E
:101320001C9FF0011D9FF00D1124E051FE4F4081E4
:10133000518162817381848195810E949E072196EB
:10134000C770E9CFDF91CF911F910895409120029E
:101350005091210260912202709123028091240217
:10136000909125020C949E07EF92FF920F931F938A
:10137000CF93DF938091250282958F7009F065C02D
:1013800080912202882309F460C08091EE01F090E0
:10139000EF011091200200912102609123027091CF
:1013A000240291E01F3F09F090E0C0910001D0912C
:1013B0000101292F96E0E92E8F1509F446C0611529
:1013C000710521F00F3F21F030E003C031E001C092
:1013D000322F90E030FD36C0E89EF001E99EF00D1E
:1013E0001124DF01A051BE4F11963C91119730138B
:1013F00029C03C91311326C012963C9112973111AD
:1014000021C013964D915C911497461B570B4C17B6
:101410005D07C0F4809125028F7080618093250262
:10142000EB50FE4F80818F708061808380E292E07C
:101430000E941C07DF91CF911F910F91FF90EF90B9
:101440000C94850901968770B7CFDF91CF911F91DA
:101450000F91FF90EF9008959F92AF92BF92CF921D
:10146000DF92EF92FF920F931F93CF93DF93CDB74D
:10147000DEB761970FB6F894DEBF0FBECDBF8C010B
:1014800085E0F801DE011D9601900D928A95E1F745
:10149000D8011296EC9090912002E09121022091C7
:1014A0002302309124022115310531F0EF3F31F450
:1014B00081E09F3F19F403C081E001C080E0B82FB4
:1014C000B1709B2E80FD47C1D8014C9111965C9163
:1014D00011971396AD90BC90149780E2C82E82E0CD
:1014E000D82EF0902202B501621B730B20910001EF
:1014F00030910101FF2009F4D9C0809125026217C3
:10150000730708F095C0282F207F09F052C05E13A2
:1015100013C0491311C0FE2CE1100EC08F70806102
:10152000809325020E94A609C6010E941C07809193
:101530002502F80185834DC1AB2831F05F3F31F4BE
:1015400081E04F3F19F403C081E001C080E080FDDD
:1015500003C081E08E2502C080E090E0F82FF1709A
:10156000FF2E80FF1CC08091EE012091EF0136E03C
:10157000821709F40BC190E0389FF001399FF00DFC
:101580001124E051FE4F6181561306C0608146135D
:1015900003C06281E61203C001968770E9CFFE2C7A
:1015A000EE2009F416C18091250281608093250206
:1015B00054C05E1306C0491304C0E11002C0F80114
:1015C00099C0C8010E948707882361F1EE2051F17C
:1015D00020912502822F82958F7090E0029774F0FF
:1015E000809120029091210298878F831986BB8673
:1015F000AA862C87CE0107960E941C0786E0F80178
:10160000A0E2B2E001900D928A95E1F70E94B40940
:101610000E94A6090AC05E1711F1C8010E9487073F
:1016200081112CC0C8010E941C07FF24F394D1C073
:10163000282F207F81F77A2DB98AA88A6E2D898973
:101640000E948F0780E292E00E941C0786E0D6018C
:101650001D928A95E9F70E94A609F12CBAC0491398
:10166000DCCFE110DACFF8018583C8010E941C07A6
:1016700086E0D6011D928A95E9F7ABC0EE2091F283
:1016800020912502822F82958F7090E002970CF4B2
:10169000B5CF80912002909121029A8389831B8289
:1016A000BD82AC822E83CE010196A6CF621773074E
:1016B00008F044C0FE2CEE2009F4B4CF5E1330C015
:1016C00049132EC02091250220FD21C0822F829532
:1016D0008F70482F50E041155105C9F0F80125835E
:1016E0004F30510541F08F5F982F9295907F822F58
:1016F0008F70892B8583C8010E941C0786E0F80142
:10170000A0E2B2E001900D928A95E1F73CC086E03C
:10171000F801A0E2B2E001900D928A95E1F759C07C
:10172000C8010E948707811169CF809125028160DD
:1017300080932502C8010E941C074BC07A2DB98AEC
:10174000A88A6E2D89890E948F0786E0D6011D9296
:101750008A95E9F718C0EE2009F464CFC8010E9409
:101760008707F82E882309F45DCF86E0F801A0E210
:10177000B2E001900D928A95E1F780E292E00E943A
:1017800015040E94B4090E94A60923C04D875E87F4
:101790008D859E850E945709292F22952F70223012
:1017A00028F49F7039F0811105C00BC0243028F453
:1017B0009F7049F4805E883020F0C8010E941C07A9
:1017C0009F2CF92C06C0D80115969C91907F91F71B
:1017D000F8CF8F2D61960FB6F894DEBF0FBECDBF48
:1017E000DF91CF911F910F91FF90EF90DF90CF90FD
:1017F000BF90AF909F9008951F93CF93DF93CDB785
:10180000DEB72C970FB6F894DEBF0FBECDBF4F8367
:10181000588769877A878B879C87CE0107960E94B5
:101820002C0A8823D1F09F8188852A853B85232B2C
:1018300031F08F3F31F481E09F3F19F403C081E024
:1018400001C080E080FD47C04F81588569857A8559
:101850008B859C850E949E073EC086E0FE013796E0
:10186000DE01119601900D928A95E1F7FF81E885DE
:101870006A857B856115710531F0EF3F31F481E0B8
:10188000FF3F19F403C081E001C080E080FD23C068
:101890002091EF0130E0C9010196877099274091AE
:1018A000EE0150E084179507F1F1F983EA837D8317
:1018B0006C8396E0929FD001939FB00D1124A051AC
:1018C000BE4FFE01319601900D929A95E1F78093FB
:1018D000EF010E94850916E08091EE019091EF01E1
:1018E000891771F1189FC001112480519E4F0E94E9
:1018F0002C0A882329F1E091EE011E9FF0011124AA
:10190000E051FE4F408151816281738184819581D4
:101910000E949E078091EE0190E0019687709927C2
:101920008093EE01D9CF0E9468071092EF011092C8
:10193000EE01E0E2F2E086E0DF011D928A95E9F730
:101940002C960FB6F894DEBF0FBECDBFDF91CF91BE
:101950001F91089580912E0285958595859508950E
:1019600080912E028770089590912E02977081E0E9
:1019700009F480E008958091390208959091390228
:10198000892B80933902089580959091390289239B
:101990008093390208951092390208959091380287
:1019A000892B80933802089580959091380289237D
:1019B00080933802089510923802089580912F0282
:1019C000089508950C94E10C0C94E20C909183021C
:1019D00092FD08C090912F02981721F080932F025A
:1019E0000C94E40C089580912F02882329F0109222
:1019F0002F0280E00C94E40C0895CF93DF93E091E4
:101A00000201F0910301809139028083E09102018B
:101A1000F0910301908180913802892B808380911D
:101A20002F02882381F0E0910201F091030190815F
:101A3000892B808380910201909103010E94761F7F
:101A400081110E94F30CC0910201D091030148E082
:101A500050E066E272E0CE010E944428892B69F0D2
:101A600088E0FE01A6E2B2E001900D928A95E1F7CE
:101A7000CE01DF91CF910C94311FDF91CF9108956A
:101A80000C94E10C9091830292FD10C098E0899F24
:101A900090011124262B20932E020E942008809171
:101AA0002E028595859585950C94400D0C94200803
:101AB00010922E0280E00C94400D20912E02809511
:101AC000822380932E02982F977099F430E0482F4C
:101AD000082E000C550B2417350759F090918302FE
:101AE00092FD07C08595859585950E9441080C94C7
:101AF000580D08959091830292FB222720F9281710
:101B000069F080FB92F99093830280918202909118
:101B100083020E94C80D82E00C945D0D08958091AF
:101B2000830282FB882780F991E089270C947A0D43
:101B300081E00C947A0D80E00C947A0D6FEF7FEFCA
:101B400080E090E00C94832880E090E00E945F2881
:101B500021E0893E9E4F09F020E0822F089582E027
:101B600090E00C94512883E090E00C945128CF939E
:101B700084E090E00E945128C82F82E290E00E9409
:101B800051282C2F30E0A901582BCA01CF9108957C
:101B9000CF93C92F682F84E090E00E9465286C2FB6
:101BA00082E290E0CF910C946528AB01BC018FE0FC
:101BB00090E00C947728AB01BC0183E190E00C9499
:101BC000772860E070E0CB010C94DB0D60E070E002
:101BD000CB010E94D50D0C94E10D69EE7EEF80E003
:101BE00090E00E94832860E082E090E00E946528F7
:101BF00060E083E090E00E9465281092EA01109274
:101C0000EB011092EC011092ED0160E084E090E0B5
:101C10000E94652860E082E290E00E94652860E012
:101C200085E090E00E94652860E086E090E00E94F8
:101C300065286FEF87E090E00E94652840E050E063
:101C4000BA0188E090E00E94772860E08DE090E0A3
:101C50000E94652840E050E0BA0188E190E00E94CF
:101C6000772860E087E190E00E94652840E050E03E
:101C7000BA018CE190E00E94772860E070E080E299
:101C800090E00E94832840E050E0BA0188E190E0B3
:101C90000E9477280C94E60D0C94ED0D682F8EE0D1
:101CA00090E00C9465280E946B206093460270932C
:101CB00047028093480290934902609342027093D6
:101CC00043028093440290934502089585B780684B
:101CD00085BF85B7806885BF089581E008950C941D
:101CE0006D0E08950C94710E0C94710E0C94740E7C
:101CF0000C94710E0C94780E0C94710E0E94660E6A
:101D00008EE391E10E941B1F0E947C0E0C947A0EC0
:101D10000E94720E0C94710E0E945B110C94AF0322
:101D20000E9456200E9440120E948C0E0E94F11ABE
:101D30000C94760E5F926F927F928F929F92AF92E9
:101D4000BF92CF92DF92EF92FF920F931F93CF93A8
:101D5000DF93CDB7DEB72A970FB6F894DEBF0FBE7C
:101D6000CDBF0E945512C82E81110E94530E3AE336
:101D7000832E32E0932E00E010E0502E802F0E9440
:101D80007F115C01F401619071904F016826792602
:101D900061147104B1F40F5F1F4F0430110569F72E
:101DA0008FEF89838A831B820E945F208160782F56
:101DB0009D838C8349815A816B818D810E94CB03E5
:101DC0003AC080914A0281FD0E948811D12CEE24F4
:101DD000E394F12CC3018E219F21892B29F10E94CC
:101DE0006F0E8823A9F0DE825F82AE20BF2081E0E3
:101DF000AB2809F480E088870E945F208160782FFB
:101E00009A8789874E815F8168858A850E94CB0386
:101E1000000F111FF801E65CFD4F80819181E826DB
:101E2000F926F182E08207C0D394EE0CFF1CFCE09F
:101E3000DF12D0CFB0CF81E0C11001C080E02A9680
:101E40000FB6F894DEBF0FBECDBFDF91CF911F91CB
:101E50000F91FF90EF90DF90CF90BF90AF909F9049
:101E60008F907F906F905F9008950E949A0E0E94CD
:101E7000351B0E945C140C94C003CF93DF930E9427
:101E80006710EC01811521E5920708F045C0811526
:101E900030E5930708F094C0883E910528F5803E10
:101EA000910508F0F8C0883A910570F4853A9105DB
:101EB00008F07CC08130910509F475C008F4E8C0D1
:101EC000049708F0E8C0E4C08F3B910508F0E0C03B
:101ED000C85AD0E0CC0FDD1FC35ADE4F0990D8811D
:101EE000C02DCE019464D8C0811540E2940758F407
:101EF000811551E0950708F0CEC08D3E910508F49C
:101F0000C7C09065C9C0C11580E4D80708F4C0C037
:101F1000DF70CE01906AC0C0811525E59207A8F454
:101F2000811534E5930708F095C0811543E59407C2
:101F300008F07BC0811552E5950708F061C0D82FE5
:101F4000CC27CE01816F906AA7C0C11589E5D8075B
:101F5000A0F4C11528E5D20708F082C0C11536E506
:101F6000D30708F095C08C2F0E94FB108F7190E072
:101F7000D82FCC27CE0190628FC0C1154AE5D40777
:101F800008F474C0CE0190568115904208F080C0CC
:101F90008D2F8F710E94FB10DD27D0628F71AE01F3
:101FA000582BCA0179C081E090E076C0C55AD0E0D4
:101FB000C557DE4F8881C82FD0E0CE0190646CC039
:101FC00074E0969587957A95E1F7282F23703C2F3A
:101FD000337081E090E002C0880F991F3A95E2F7D4
:101FE0009C68AC01522B9A019C2F9F7096959695F8
:101FF00050E2959FE0011124C9018C2B9D2B4CC010
:102000008370992721E030E002C0220F331F8A95A8
:10201000E2F79C2F9695969580E2989FE001112417
:10202000C22BD32BCE019C6837C08370992721E047
:1020300030E002C0220F331F8A95E2F79C2F96955D
:10204000969540E2949FE0011124C22BD32BCE0140
:102050009A6822C0D82FCC27CE01846F906A1CC00A
:10206000DC2FCC27CE01806F906A16C08C2F8F702A
:102070000E94FB1094E0D695C7959A95E1F7CF7032
:10208000D0E0DC2FCC27D0699E01282BC90104C0E9
:1020900080E090E001C0CE01DF91CF91089520E370
:1020A000829FC0011124FC012CE0729FE00DF11D04
:1020B0001124E60FF11DEE0FFF1FE852FF4F85912F
:1020C000949108950E944F100E943D0F0895823808
:1020D000910569F1B0F48133910509F46DC048F4BC
:1020E0008932910509F463C08A32910509F469C007
:1020F00008958533910509F455C089339105B9F0E8
:102100000895833E910569F138F4803E9105B1F060
:10211000823E910509F10895863E9105A9F1873E19
:102120009105B9F1843E910509F064C023C0209166
:10213000820220FD4FC021FD4DC008958091820292
:1021400080FD44C08091830280FF44C08091820260
:1021500084FD42C083EE4DC08091820282FF38C070
:10216000F5CF8091820282FD33C08091830280FD91
:1021700031C0ECCF8091830281FF32C08091820216
:1021800084FD2AC087EE35C08091820283FF26C07D
:10219000F5CF8091820283FD21C08091830281FD71
:1021A0001FC0ECCF8091820285FD1CC01DC08091B4
:1021B000820285FD19C016C08091820286FD16C07C
:1021C00017C08091820286FD13C010C089E311C040
:1021D00082EE0FC080EE0DC080E00BC086EE09C01D
:1021E00084EE07C089E205C085E303C08AE201C02E
:1021F00081E390E008959091820292FF0DC0282F14
:102200002871283019F4877F846006C0282F247134
:10221000243011F48B7F886093FF0DC0282F287124
:10222000283119F4877E846106C0282F2471243157
:1022300011F48B7E88612091830220FF0DC0382F1E
:102240003871383019F4877F816006C0382F3171BA
:10225000313011F48E7F886021FF0DC0282F287146
:10226000283119F4877E816106C0282F2171213120
:1022700011F48E7E886194FD877E089580E0089534
:102280000C949E0D0E9455122FEF86E791E021508D
:1022900080409040E1F700C000000E94551280E0AD
:1022A0000E947F1180FF04C00E9440110C94AC205A
:1022B00008950C9442110E94A40D811102C00E9445
:1022C0004C0E0E94AF0D80934A020E94B70D90936E
:1022D0008302809382020E9459110E94B30D682FDD
:1022E00070E080E090E00E94C0076091E60170918C
:1022F000E7018091E8019091E9010C94F807E82F3B
:10230000F0E0EE0FFF1FE457FD4F808191810895AB
:10231000089580EA8A95F1F7089500C008950C9415
:10232000891108950C9491110C9492110C949111AF
:102330000C949611F894E82FE295EF70F0E031A13B
:10234000282F2F7081E090E001C0880F2A95EAF7CE
:10235000982F9095932391A392A1892B82A378948F
:1023600008950F931F93CF93DF93CAE9D1E089912A
:102370008F3F11F00E949A1181E0CE39D807B9F74A
:10238000CEE8D1E00AE911E089918F3F11F00E9477
:102390009A110C171D07C1F7DF91CF911F910F9173
:1023A0000895BF92CF92DF92EF92FF920F931F9307
:1023B000CF93DF938C01C62FD0E0CE0186569E4F7F
:1023C0006C01FC0190819F3F09F450C0B62EF89437
:1023D000E92FE295EF70F0E081A19F7021E030E0FD
:1023E00001C0220F9A95EAF7822B81A382A1209542
:1023F000282322A378940E948D11EEE8F1E04AE9A7
:1024000051E021E030E0E12CF12C61916F3F89F047
:10241000A62FA295AF70B0E090968C9190E06F706F
:1024200002C0959587956A95E2F780FD02C0C901C3
:1024300002C080E090E0E82AF92A220F331F4E17ED
:102440005F0719F7F60180818F3F11F00E949A1102
:1024500061E0E114F10409F460E08B2D0E948F111A
:10246000CC0FDD1FC00FD11FF982E882DF91CF9121
:102470001F910F91FF90EF90DF90CF90BF90089544
:102480000E94B11188E0ECE8F2E0DF01982F1D9284
:102490009A95E9F7E4E8F2E0DF011D928A95E9F701
:1024A00084E00E94A0120C942F03FF920F931F93BD
:1024B000CF93DF93CDB7DEB728970FB6F894DEBF82
:1024C0000FBECDBF8E010F5F1F4F88E0F801119244
:1024D0008A95E9F7F12C6F2DC8010E94D111F39470
:1024E000F4E0FF12F8CF48E050E0B80184E892E051
:1024F0000E944428FF24F394009709F4F12C892BBF
:1025000041F088E0F801A4E8B2E001900D928A95CC
:10251000E1F72F2D44E06CE872E084E892E00E943D
:10252000A1120E9431038F2D28960FB6F894DEBFBA
:102530000FBECDBFDF91CF911F910F91FF900895F6
:102540000895FF920F931F93CF93DF93F82E092FD7
:10255000162FD72FC42F222349F081E080934D02FC
:102560000E945F2090934C0280934B0280914D0219
:102570008823D9F080914B0290914C020E947720E1
:10258000059798F0EF2DF02FA12FBD2F80E090E060
:102590004C2F50E08417950734F4219131912D93FD
:1025A0003D930196F7CF10924D02DF91CF911F918D
:1025B0000F91FF9008950E9462220E94900E0C9449
:1025C0006E220E9472220E94350F0C948C220E946F
:1025D000FD1F0E9449220E947E0E0E94DB120E9473
:1025E000E1120E94880EFBCF8091540280FF06C04A
:1025F0006091090170E0660F771F26C081FF04C05B
:102600006091090184E005C082FF07C06091090163
:1026100088E0689FB001112417C09091530299235C
:10262000D1F060910801961788F72091090188E0A0
:10263000289F90011124929FA001939F500D112477
:1026400070E0CA010E94BE276038710540F4611530
:10265000710519F406C068E070E0862F08958FE7D1
:10266000089581E008958091540280FF08C0609130
:10267000050170E0759567957595679521C081FF97
:1026800006C06091050170E07595679519C082FFDD
:1026900004C06091050170E010C09091520299232E
:1026A00099F0609104019617A0F780910501899F28
:1026B000C001112470E00E94BE276038710540F40B
:1026C0006115710519F406C061E070E0862F089568
:1026D0008FE7089581E008958D3E21F40E94F41261
:1026E000819504C08E3E29F40E94F4128093580212
:1026F00008958F3E21F40E94F412819504C0803F1A
:1027000029F40E94F412809357020895893F19F426
:102710000E94331305C08A3F31F40E943313819520
:102720008093590208958B3F21F40E9433138195C1
:1027300004C08C3F29F40E94331380935A020895F9
:102740009FE0980F983078F421E030E0A90102C0B2
:10275000440F551F9A95E2F7CA0190915602892BB2
:102760008093560208958D3F21F480915402816038
:102770000BC08E3F21F480915402826005C08F3FD0
:1027800029F48091540284608093540208958D3E10
:1027900039F49091580297FF35C01092580259C0F1
:1027A0008E3E29F4909158021916BCF32BC09091DB
:1027B00057028F3E29F497FF25C01092570249C057
:1027C000803F19F41916CCF31DC090915902893F2E
:1027D00029F41916BCF4109259023BC08A3F19F42F
:1027E00097FF10C0F8CF8B3F39F490915A0297FFB2
:1027F00009C010925A022DC08C3F21F490915A02C8
:102800001916BCF39FE0980F983080F421E030E077
:10281000A90102C0440F551F9A95E2F7CA0180959D
:102820009091560289238093560213C08D3F21F464
:10283000809154028E7F0BC08E3F21F48091540210
:102840008D7F05C08F3F29F4809154028B7F809348
:10285000540280915702811106C080915802811163
:1028600002C01092530280915902811106C08091DA
:102870005A02811102C01092520208950E945F20F4
:1028800020915702211104C020915802222321F0E7
:10289000909351028093500220915902211104C05B
:1028A00020915A02222321F090934F0280934E02EE
:1028B00085E592E00C943C1FEF92FF920F931F93DB
:1028C000CF93DF9300D000D000D0CDB7DEB786E045
:1028D000E5E5F2E0DE01119601900D928A95E1F7AF
:1028E000E0905702F09058020091590210915A025C
:1028F00010925702109258021092590210925A02E6
:10290000E11003C0FF2009F45DC080915002909156
:1029100051020E947720AC0190915302992339F023
:1029200020910A0130E02417350758F04BC0209160
:102930000B018AE0289F900111242417350718F015
:1029400041C09F3F19F09F5F90935302EE2061F0CA
:102950000E94F4121E1414F09FEF01C091E0989FA2
:10296000902D112490935702FF2061F00E94F412E1
:102970001F1414F09FEF01C091E0989F902D112437
:1029800090935802309157023323E1F0209158027E
:102990002223C1F045EB3403C0011124992319F01F
:1029A0009093570203C081E08093570235EB2303D5
:1029B000C0011124992319F09093580203C081E0BB
:1029C00080935802011103C0112309F45DC0809166
:1029D0004E0290914F020E947720AC0190915202DA
:1029E000992339F02091060130E02417350758F07B
:1029F0004BC0209107018AE0289F900111242417E1
:102A0000350718F041C09F3F19F09F5F9093520225
:102A1000002361F00E943313101614F09FEF01C0E1
:102A200091E0989F902D112490935902112361F009
:102A30000E943313111614F09FEF01C091E0989F8C
:102A4000902D112490935A02309159023323E1F0D2
:102A500020915A022223C1F045EB3403C001112416
:102A6000992319F09093590203C081E08093590291
:102A700035EB2303C0011124992319F090935A02D6
:102A800003C081E080935A028091570281110BC0EC
:102A900080915802811107C080915902811103C0B1
:102AA00080915A0281110E943E14EB82FC820D83B8
:102AB0001E8386E0FE013196A5E5B2E001900D92FD
:102AC0008A95E1F726960FB6F894DEBF0FBECDBF0C
:102AD000DF91CF911F910F91FF90EF900895E5E561
:102AE000F2E086E0DF011D928A95E9F71092530229
:102AF00010925202109254020895EF92FF920F9397
:102B00001F93CF93DF938B01682F11110AC04423C9
:102B100029F0E82FF0E0E15FFC4F6491762F862FDB
:102B200075C0212F30E0E82FF0E0442321F0E15F71
:102B3000FC4FE491F0E046E0049FC0011124CFEF88
:102B4000D0E0BE010E94AA274BEA4603C001479F7E
:102B5000900D1124800F911D800F911D982F990FBA
:102B6000890FAE01421B530B4E9FD0014F9FB00DFA
:102B70005E9FB00D11249B2F189FA0011124452F9B
:102B800055278E01041B150B0E9FA0010F9F500DA2
:102B90001E9F500D11247E01E81AF108E29E80016B
:102BA000E39E100DF29E100D1124212F3327C21B1E
:102BB000D30BCE9F9001CF9F300DDE9F300D11249F
:102BC00062307105A9F048F46115710569F0613052
:102BD0007105C9F48B2F752F0DC06430710581F01C
:102BE00058F06630710579F47E2F8B2F932F0DC02E
:102BF000832F7B2F9E2F09C08E2F7B2F952F05C0F3
:102C00008E2F732F02C07E2F852F692FDF91CF91DA
:102C10001F910F91FF90EF90089541E00E947D1564
:102C2000089508950E940D160895CF93DF93762F8F
:102C3000E901682F842F0E941216798368838A83A2
:102C4000DF91CF91089580919402282F269530E04E
:102C50002115310519F48170826005C025323105D6
:102C600024F08170886480939402089588E090E055
:102C70000C945928CF92DF92EF92FF926B017C0166
:102C80000E942316B701A60188E090E0FF90EF9024
:102C9000DF90CF900C947728E4E9F2E083E0808322
:102CA00011828FEF8283838314826081718182819C
:102CB00093810C943A168091940280FF02C086950D
:102CC000089580E0089590919802933018F49F5FE2
:102CD00090939802882351F060919402709195022C
:102CE00080919602909197020C943A16089581E093
:102CF0000C94631690919802992319F09150909337
:102D00009802882351F0609194027091950280910D
:102D10009602909197020C943A16089581E00C94D3
:102D20007A1670E00C94B21C6091100180919402AC
:102D300080FF0AC080910F0123E0829FC00111240F
:102D400087569D4F0C94911680911101909112011C
:102D5000891780F7E82FF0E09F01220F331FE20F61
:102D6000F31FE756FD4F1182108212828F5FF0CF62
:102D70009091940290FF16C0909111012091120140
:102D8000921770F4E92FF0E0DF01AA0FBB1FEA0FE2
:102D9000FB1FE756FD4F8183608342839F5FF0CF27
:102DA0000C9494160895CF93DF9300D01F92CDB763
:102DB000DEB79091940290FF0AC09E012F5F3F4FB3
:102DC0000E9415164B8169818A810E94B8160F9066
:102DD0000F900F90DF91CF910895CF93DF93EC0187
:102DE000EC81F0E0E65FFD4F4491E4E9F2E06281BE
:102DF00081810E94D3168C818F5F8C83DF91CF916C
:102E00000895CF93DF93EC01E4E9F2E0438162811E
:102E10008C810E94D3168C818F5F8C83DF91CF9140
:102E200008950F931F93CF93DF9300D01F92CDB7D8
:102E3000DEB78C0180915B0281110AC09E012F5F79
:102E40003F4F4FEF6FEF0E9415168A8180935B0210
:102E5000F8018481813051F028F0823061F4409192
:102E60005B020AC080915B0240E007C060915B0298
:102E700040E080E003C040E080E060E00E94B816DF
:102E8000F801848190E0019663E070E00E94BE2723
:102E900084830F900F900F90DF91CF911F910F912E
:102EA0000895AF92BF92CF92DF92EF92FF920F936D
:102EB0001F93CF93DF9300D01F92CDB7DEB7182FAB
:102EC000F62E042FE22E9091940290FF6DC0E92F10
:102ED000E695AE2FB0E0A256BE4F8C91809367026C
:102EE0009E7F923061F49E012F5F3F4F812F0E94A1
:102EF00015164B8169818A810E94B81643C08230C1
:102F000019F4009197023EC0863019F41091950291
:102F100039C08930D9F38931A9F5E9518E2F8170F3
:102F2000D82EE695F0E0E65FFC4FA590B490C12C5A
:102F3000BB2460911301C61618F52C2D30E0A29E1B
:102F4000C001A39E900DB29E900D112470E00E94CE
:102F5000AA27812FD11002C0860F01C0861B909135
:102F60001101290F311DA901440F551F240F351FD1
:102F700027563D4F402F6F2D0E941516C394D9CF71
:102F80000E94941610939502F09296020093970275
:102F9000EE2051F06091940270919502809196021A
:102FA000909197020E943A160F900F900F90DF9128
:102FB000CF911F910F91FF90EF90DF90CF90BF9036
:102FC000AF900895E4E9F2E09181282F4381628176
:102FD00088E0890F0C94511781E00C94E217E4E922
:102FE000F2E09181282F4381628188EF890F0C9450
:102FF000511781E00C94EF17E4E9F2E0628121E1DE
:10300000620F08F46FEF282F438181810C945117D0
:1030100081E00C94FC17E4E9F2E0628121E1621B9B
:1030200008F460E0282F438181810C94511781E0DE
:103030000C940B18E4E9F2E0438121E1420F08F41B
:103040004FEF282F628181810C94511781E00C94FD
:103050001A18E4E9F2E0438121E1421B08F440E060
:10306000282F628181810C94511781E00C942918DA
:1030700020E00C945117FF920F931F93CF93DF938F
:10308000EC01F12C0FEF10E060911301F616F0F453
:10309000809111012F2D30E0280F311DC901880FBB
:1030A000991F280F391F27563D4F70E0C8010E9415
:1030B000BE27962F8C814091970260919602F99ECF
:1030C000800D11240E941516F394DECF0E949416F1
:1030D0009A818C8190FF02C08F5F01C081508C83E8
:1030E000DF91CF911F910F91FF900895AF92BF9202
:1030F000CF92DF92EF92FF920F931F93CF93DF93C4
:10310000FC01828180FF02C00FEF01C001E010E0EE
:103110004DE0A42E80911301181708F043C0809150
:103120001101C12ED12CE601C80FD11DCE01880F8F
:10313000991FC80FD91FC756DD4F198218821A82EE
:1031400034E0E32EF12CB12C80915D028B0D8E309A
:103150002CF06A2D0E949C27892F05C087FF03C091
:1031600090911301890F082E000C990BC816D906EF
:1031700091F4809197028E9DA0018F9D500D112496
:1031800055954795559547959E016091960280917A
:1031900095020E941516B00EF1E0EF1AF108A1F6A3
:1031A0001F5FB8CF0E94941680915D02013031F408
:1031B000811102C080911301815007C090E00196F7
:1031C0006091130170E00E94BE2780935D02DF9141
:1031D000CF911F910F91FF90EF90DF90CF90BF9014
:1031E000AF900895CF9380911101909112018917AA
:1031F00070F4E82FF0E09F01220F331FE20FF31F5E
:10320000E756FD4F1182108212828F5FF0CFC0E02F
:1032100060911301C617C0F5EC2FF0E070E0CF010C
:103220000E94BE2720911101820F20915C02022E84
:10323000000C330B90E0E217F307CCF020910E0165
:10324000022E000C330B2E173F078CF09C01220F2F
:10325000331F820F931F9C0127563D4F40919702C9
:1032600060919602809195020E9415160BC0FC0198
:10327000EE0FFF1F8E0F9F1FFC01E756FD4F1182BF
:1032800010821282CF5FC4CF0E94941620910D014C
:1032900080915C02820F80935C0290910E01920FEC
:1032A00090930E0119165CF4082E000C990B4091B6
:1032B000130150E041505109841795071CF02195E6
:1032C00020930D01CF9108958F929F92AF92BF925C
:1032D000CF92DF92EF92FF920F931F93CF93DF93E2
:1032E0008C01FC014481C42FD0E09E01DE010E94CC
:1032F00002289B01AC010E9418286B017C01E0E2CE
:10330000F0E0EC1BFD0BA5E5B0E09B01AC010E94D9
:1033100018284B015C019F01DF010E94FA279B01E5
:10332000AC010E9423289B01AC012C0D3D1D4E1DBC
:103330005F1DC501B4010E94D227C22FD22F2A32AD
:1033400028F4F3E02F9F900111240DC025E530E013
:103350002C1B3109C901880F991F280F391F37FF0E
:1033600002C02F5F3F4F35952795C22FC095F12C96
:1033700085E5E82EED1A80911301F816C8F4F1FCEA
:1033800002C08E2D01C08D2F909111012F2D30E0A4
:10339000290F311DA901440F551F240F351F275632
:1033A0003D4F4C2F609196020E941516F394E3CF87
:1033B0000E949416F8018481811102C091E003C03B
:1033C000803219F49FEF90930C0190910C01890FBA
:1033D000F8018483DF91CF911F910F91FF90EF90BF
:1033E000DF90CF90BF90AF909F908F9008950F93F4
:1033F0001F93CF93DF93EC0100E010E08091130165
:10340000282F30E00217130724F59091110198013D
:10341000290F311DA901440F551F240F351F2756B1
:103420003D4F869590E04C81081719071CF4442302
:1034300031F002C0411103C04091970201C040E049
:1034400060919602809195020E9415160F5F1F4FA2
:10345000D5CF0E9494168C8190E0019681709927B7
:103460008C83DF91CF911F910F910895E4E9F2E0F1
:1034700080818E7F808360817181828193810E94AF
:103480003A16109268022FEF80E792E021508040B8
:103490009040E1F700C000000C949416E4E9F2E0DB
:1034A00080818E7F8083109268022FEF80E792E008
:1034B000215080409040E1F700C000000C94941629
:1034C000109268028091650281110AC081E08093A8
:1034D0006502809194028170809364020C944E1A6C
:1034E000089560919402669570E04BE050E084E1AD
:1034F00091E00E943728892B19F481E080936802BB
:103500000E945F2090935F0280935E0208959091E5
:10351000940290FF35C09170811102C0926006C084
:10352000853210F0986402C0880F982B9093940213
:10353000662351F0609194027091950280919602F9
:10354000909197020E943A1660919402669570E0FD
:103550004BE050E084E191E00E943728892B19F07C
:103560001092680202C00E94711A81E08093610289
:103570004091970260919602809195020C943818C0
:103580000895682F90919402969581E0890F853275
:1035900008F081E00C94871A81E00C94C11A682F1E
:1035A0009091940296958FEF890F09F484E20C9420
:1035B000871A81E00C94CF1A61E00C94871AE4E931
:1035C000F2E080818160808386950C94DC1A809182
:1035D000940280FD0C94361A0C94DF1A60E00C946F
:1035E000871A8091660281112EC00E94A40D81115C
:1035F00004C00E944C0E0E944C160E943616609326
:1036000094027093950280939602909397026E7F36
:1036100061F40E944C160E943616609394027093D7
:10362000950280939602909397020E94231610921F
:1036300068028091940280FF03C086950E94EE1A72
:1036400081E0809366020895E4E9F2E08081816080
:10365000808386950C94EE1A109265028091640224
:1036600081110E94241B0C94711A0F931F93CF9306
:10367000DF9380916802882309F485C080916702F6
:10368000E0919402E695E81BE0936002823049F4F1
:10369000F0E0EA5FFD4FE491CE2FD0E00DEE16E1B1
:1036A00049C0863049F4F0E0ED5FFD4FE491CE2F44
:1036B000D0E001E017E13EC0893051F4E695F0E03A
:1036C000E050FE4FE491CE2FD0E00BE318E132C082
:1036D0008F3051F4E695F0E0E350FE4FE491CE2FA9
:1036E000D0E006E718E126C0853149F4F0E0E65065
:1036F000FE4FE491CE2FD0E002EF18E11BC08831DD
:1037000081F0833239F4E8EFF1E0C591D49101E121
:1037100017E110C0843251F4C4EFD1E007EF19E192
:1037200009C0C8E2D0E004E619E104C0C0EDD7E06A
:1037300001E116E180916102882361F0109261023B
:103740000E945F2090935F0280935E02109263025A
:10375000109262020E945F20E0915E02F0915F028F
:103760008E1B9F0B8F3F9F4770F4EC0FFD1FF09354
:103770005F02E0935E028EE592E0F801DF91CF9167
:103780001F910F910994DF91CF911F910F9108958F
:10379000882311F0FA0101C0FB010994CF93DF9354
:1037A000C82FD62F0E945B168C1740F00E945B1624
:1037B0008D1720F4DF91CF910C94CC1A8C2FDF91D0
:1037C000CF910C94DC1A1F93CF93DF93FB011281EE
:1037D0001111C3C0EC010E94BB0C8272CD3CFCE510
:1037E000DF0709F49AC0A8F5C73CECE5DE0709F449
:1037F00076C0A8F4C43C9CE5D90709F45FC028F45E
:10380000C33CDC4509F457C054C0C53C9CE5D9070E
:1038100009F459C0C63CDC4509F45CC04AC0CA3C46
:10382000FCE5DF0709F46AC050F4C83CECE5DE07AC
:1038300009F45AC0C93CDC4509F45BC03AC0CB3C32
:103840009CE5D90709F45FC0CC3CDC4509F460C0B5
:1038500030C0C23DFCE5DF0709F46FC088F4CF3CFF
:103860009CE5D90709F460C008F45CC0C03DFCE5E4
:10387000DF0709F45CC0C13DDC4509F45BC019C039
:10388000C53D9CE5D90709F460C050F4C33DFCE593
:10389000DF0709F455C0C43DDC4509F454C009C034
:1038A000C63D9CE5D90709F455C0CE35DD4509F480
:1038B00054C011E052C00E94E71A4FC049ED5AE1CE
:1038C0006CEC7AE104C04CEC5AE169ED7AE10E94BB
:1038D000C81B43C049EF57E16CEE77E1F8CF4CEEDF
:1038E00057E169EF77E1F3CF47E158E168E078E12C
:1038F000EECF48E058E167E178E1E9CF45E358E1F0
:1039000066E278E1E4CF46E258E165E378E1DFCFB3
:103910004EE856E167E776E1DACF47E756E16EE831
:1039200076E1D5CF81E017C065E082E010C068E0A5
:1039300086E00DC06EE089E00AC064E18FE007C058
:1039400067E185E104C088E106C062E289E10E9486
:10395000CE1B03C083E20E94DC1A812FDF91CF913E
:103960001F9108956E9A2EB12F7B3EB130644FB7F0
:10397000F894FC01CB01880F991F680F791F6E0F17
:103980007F1FE617F70789F0819198E03EB90000A4
:1039900000C087FF2EB9880F000000C000C000C023
:1039A0002EB900C09A9591F7ECCF4FBF8FE594E008
:1039B0000197F1F700C000000895CF93DF93EC0169
:1039C000FB018281882309F43CC1C430FDE5DF0797
:1039D00060F4CB3F9CE5D90788F49E0122503C451A
:1039E0002431310508F02EC109C0C236EDE5DE07ED
:1039F00029F0C63AFDE5DF0709F024C10E94B70DA2
:103A00009093830280938202C1318CE5D80709F438
:103A1000C6C008F042C0C930ECE5DE0709F49BC01F
:103A200000F5C5308CE5D80709F485C078F4C330BB
:103A3000ECE5DE0709F478C008F07AC0C230DC4556
:103A400009F0F5C0809182028160EFC0C7309CE52B
:103A5000D90709F478C008F07AC0809182028061A9
:103A6000E4C0CD30FCE5DF0709F487C058F4CB3063
:103A70009CE5D90709F479C008F07BC080918202E7
:103A800088606FC0CF30FCE5DF0709F480C008F024
:103A900082C080918202877FC8C0CE3F9CE5D90753
:103AA00009F471C000F5C531FCE5DF0709F485C0F4
:103AB00068F4C3319CE5D90709F475C008F095C0D6
:103AC0000E946807809182028F77AFC0CC3FFCE5EF
:103AD000DF07A9F108F054C0CB3FDC4509F0A7C0CF
:103AE0008091830240C0C230EDE5DE0709F489C051
:103AF00058F4C1158DE5D80709F45AC008F069C01B
:103B00008091830282602FC0C236EDE5DE0709F4A2
:103B10007CC0C63AFDE5DF0709F481C0C330DD454E
:103B200009F085C080E06EC08091820282607DC015
:103B30008091820216C080918202886076C0809156
:103B4000830282604FC08091820280626EC0809149
:103B5000820280646AC00E94680780918202806845
:103B600064C0846062C081603DC0809182028E7FAB
:103B70005CC0809182028D7F58C08091820216C005
:103B80008091830218C0809183028D7F2BC0809129
:103B900082028F7E4AC0809182028F7D46C08091D2
:103BA00082028F7B42C080918202877F8B7F3DC0E3
:103BB000809183028D7F8E7F15C08091820282FB6F
:103BC000222720F991E0922790FB82F990FB83F95C
:103BD0002CC080918302982F909591708E7F892BB5
:103BE00090FB81F98093830222C00E946807809134
:103BF000820287FB222720F991E0922790FB87F928
:103C000014C081E00E944E0E12C08091820284FB9B
:103C1000222720F991E0922790FB84F906C0809139
:103C20008202982F909590FB80F980938202809178
:103C30008202909183020E94C80D0E94680780E072
:103C400001C081E0DF91CF910895CF93DF9386315A
:103C50009C4541F5EB010E94BB0C982F8A81209175
:103C6000020130910301882379F09A7A81E009F406
:103C700080E080936902911102C069E201C065E3AE
:103C8000C9010E94B81F0AC080916902811102C057
:103C900069E201C065E3C9010E94BA1F0E94FD0CE0
:103CA00080E001C081E0DF91CF9108950F931F93D1
:103CB000CF93DF93C42FD22FFC0182818823C9F0D8
:103CC00040936C020E945F2090936B0280936A0283
:103CD00080E28C0F883008F057C0C77081E001C0C7
:103CE000880FCA95EAF7DF91CF911F910F910C943D
:103CF000C50480916C02481330C080916A02909193
:103D00006B020E947720883C910538F510E21D0F68
:103D1000CD17B9F080E28C0F883040F4C77081E095
:103D200001C0880FCA95EAF70E94CC04183028F524
:103D300081E09D2F977001C0880F9A95EAF70E9445
:103D4000C504802F0E94BC041830F0F4D77081E0C5
:103D500001C0880FDA95EAF70AC080E28C0F88303C
:103D600098F4C77081E001C0880FCA95EAF7DF9127
:103D7000CF911F910F910C94CC04802FDF91CF91A4
:103D80001F910F910C94BC04DF91CF911F910F9163
:103D900008950F939C01CB01243F4CE5340731F18A
:103DA00088F4293DFCE53F07D9F02A3D4CE534076E
:103DB00079F1283D3C45A9F506E221EE41EE68ED9A
:103DC0007CE52BC0263FFCE53F07E1F0A8F0273F4C
:103DD0003C4539F507E225EE46EE67EF7CE51DC070
:103DE00007E225EE45EE69ED7CE517C006E221EE1F
:103DF00040EE64EF7CE511C007E225EE44EE65EF8E
:103E00007CE50BC006E221EE42EE66EF7CE505C0E4
:103E100008E221E045EE6AED7CE50E94561E80E056
:103E200008C0FC018281882319F010926C0201C045
:103E300081E00F9108959093C5018093C401089586
:103E400090937202809371020895E0917102F09153
:103E50007202309721F00190F081E02D099480E00A
:103E60000895E0917102F0917202309721F0028082
:103E7000F381E02D09940895E0917102F0917202AE
:103E8000309739F022E0DC012C930480F581E02D9D
:103E90000994089520916F02309170022817390714
:103EA00071F09093700280936F02E0917102F09133
:103EB0007202309721F00680F781E02D0994089571
:103EC00020916D0230916E022817390771F090939E
:103ED0006E0280936D02E0917102F0917202309750
:103EE00021F00084F185E02D09940895FC013296BB
:103EF00097E080E0915029F021912223D9F38F5F40
:103F0000F9CF0895662349F0FC0132960896219175
:103F1000621729F0E817F907D1F780E0089581E0EA
:103F200008959C01FC0132969FEF80E04191461775
:103F300089F09F3F19F4411101C0982F8F5F86309F
:103F4000A9F79F3F39F0F901E90FF11D97FDFA95A7
:103F50006283089508959C012A5F3F4FFC014281CE
:103F6000461301C01282019682179307B9F708958C
:103F70000C94911F0C94AB1F029626E0FC01119249
:103F80002A95E9F7089508950C94C31F83E0809360
:103F900073020C94C41F811102C081E001C082E051
:103FA000809373020C94C41F0C94CB1F81E0809308
:103FB00073020C94C41F0C94D61F08950C94DD1F3B
:103FC0000C94DE1F0C94DD1F0C94DD1F0C94DD1F80
:103FD000CF930E94E41F0E9455120E94E21FC0E08E
:103FE0008C2F0E947F11892B29F4CF5FC430C1F739
:103FF00080E001C081E0CF91089508951F920F9253
:104000000FB60F9211248F939F93AF93BF9380911C
:104010007402811113C08091C0029091C102A091DD
:10402000C202B091C3024196A11DB11D8093C0028E
:104030009093C102A093C202B093C302BF91AF910B
:104040009F918F910F900FBE0F901F9018958091A8
:10405000C802843031F10E949C031092740220E463
:1040600088E190E00FB6F894A895809360000FBEA9
:104070002093600083B7817F846083BF83B78160B2
:1040800083BF7894889583B78E7F83BF0FB6F894EB
:10409000A895809160008861809360001092600014
:1040A0000FBE08950E9468070C94A20382E084BDAD
:1040B00093E095BD9AEF97BD80936E0008952FB75A
:1040C000F8948091C0029091C102A091C202B09177
:1040D000C3022FBF08952FB7F8946091C00270916A
:1040E000C1028091C2029091C3022FBF08959C012A
:1040F0004FB7F8948091C0029091C102A091C20282
:10410000B091C3024FBF821B930B089578941F9206
:104110000F920FB60F9211248F939F93AF93BF937B
:104120008091C0029091C102A091C202B091C302DD
:104130000196A11DB11D8093C0029093C102A0936E
:10414000C202B093C302BF91AF919F918F910F9024
:104150000FBE0F901F90189581E08093E00080E2E1
:104160008093D8001092C9008FE19EE40197F1F787
:1041700000C0000087E090EBDC018093D1029093B7
:10418000D202A093D302B093D4029CE088E10FB690
:10419000F894A895809360000FBE90936000FFCFC5
:1041A000809180020895089522E02093E9002FEF86
:1041B0003091E800215035FD06C035ED3A95F1F714
:1041C00000002111F5CF2091E80025FF0BC040E051
:1041D00050E066E070E00E94FE228091E8008E7759
:1041E0008093E8000895CF93DF9321E02093E900C6
:1041F0002FEF3091E800215035FD06C035ED3A959E
:10420000F1F700002111F5CF2091E80025FF14C03F
:10421000EC0140E050E068E070E00E94FE228091F6
:10422000E8008E778093E80088E0FE01A8E7B2E01E
:1042300001900D928A95E1F7DF91CF9108958093D7
:10424000750270937702609376028091C802843081
:1042500001F582E08093E9008FEF9091E8008150B2
:1042600095FD06C095ED9A95F1F700008111F5CF07
:104270008091E80085FF0DC040E050E063E070E011
:1042800085E792E00E94FE228091E8008E7780937D
:10429000E8000895BC0184E00C941F21BC0183E078
:1042A0000C941F218091C702811109C00E948F24A4
:1042B0000E94EC248091E20084608093E2000895E3
:1042C0001092C70208950C94DB1F6091C40281E034
:1042D000611101C080E00C94C61F9091C80281E07A
:1042E000943009F080E06091C4020C94CB1F42E04E
:1042F00061EC81E00E94082442E261EC82E00E94CD
:1043000008249091C80281E0943009F080E0609127
:10431000C4020C94D41F8091CA02833009F461C096
:1043200030F4813071F0823009F49AC008958A30F7
:1043300009F486C08B3009F46CC0893009F0A8C03C
:1043400020C08091C902813A09F0A2C08091E800A2
:10435000877F8093E8008091CD029091CE02892BD7
:1043600021F468E088E792E003C060E080E090E03C
:1043700070E00E9449238091E8008B778093E800E9
:1043800008958091C902813209F082C08091CD02E6
:104390009091CE02029708F07BC08091E800877F61
:1043A0008093E8008091E80082FD05C08091C802FA
:1043B0008111F8CF6DC02091F3008091F20090E060
:1043C000922B029731F48091F100813011F0863008
:1043D00021F48091F100809380028091E8008B7736
:1043E00053C08091C902813A09F052C08091CD0238
:1043F0009091CE02892B09F04BC08091E800877F15
:104400008093E8008091E80080FFFCCF80912B0131
:1044100036C08091C9028132D9F58091CD02909148
:10442000CE02892BA9F58091E800877F8093E80070
:104430000E943D248091CB0280932B010C9468074D
:104440008091C902813221F58091E800877F8093B5
:10445000E8000E943D248091CC028093810208955F
:104460008091C902813AA1F48091E800877F80930E
:10447000E8008091E80080FFFCCF8091810280936A
:10448000F1008091E8008E778093E8000C943D2441
:10449000089584B7877F84BF0FB6F894A89580915C
:1044A0006000886180936000109260000FBE90E011
:1044B00080E80FB6F89480936100909361000FBE7E
:1044C0000C94D61F0E948F240E94EC24E2EEF0E0B0
:1044D00080818460808378940C9481278FE191E0BF
:1044E0000C94201F8091C8028530A9F48091C802E5
:1044F000853079F40E9427208091C6028823B1F389
:104500000E94E81F882391F30E94E8220E94680716
:10451000EDCF0C945220089508950C948F22292FEA
:10452000332723303105C9F060F42130310581F0A3
:104530002230310509F044C08BE390E02DE334E0F4
:1045400043C021323105E1F02232310549F138C052
:1045500082E190E028E734E037C099278130910567
:1045600049F028F0029761F5EFE0F4E005C0E9E3D7
:10457000F4E002C0EBE1F4E0849190E09F0124C0FC
:104580006115710541F061307105D1F489E090E069
:1045900028E634E019C089E090E02FE434E014C04C
:1045A0006115710541F06130710551F48BE790E0C0
:1045B0002AE834E009C080E490E025E035E004C05A
:1045C00080E090E020E030E0FA013183208308951C
:1045D00080E189BD82E189BD09B400FEFDCF8091F3
:1045E000D8008F7D8093D8008091E0008260809316
:1045F000E0008091E00081FDFCCF0895CF92DF9232
:10460000EF92FF920F931F93CF93DF93EC018B01F7
:104610007A010E945C24811133C0E114F10439F065
:10462000F70180819181081B190BC80FD91FC12C7C
:10463000D12C0115110519F18091E80085FD16C0F6
:104640008091E8008E778093E800E114F10449F04E
:10465000F70180819181C80ED91ED182C08285E088
:104660000FC00E945C24882321F30AC089918093A3
:10467000F10001501109FFEFCF1ADF0ADACF80E015
:10468000DF91CF911F910F91FF90EF90DF90CF902E
:1046900008952091CF023091D0022617370748F0B5
:1046A0006115710539F42091E8002E772093E80018
:1046B00001C0B901FC0120E06115710579F180911B
:1046C000C8028823F1F18530F1F18091E80083FD83
:1046D0003CC08091E80082FD2EC08091E80080FF00
:1046E000EBCF2091F3008091F20090E0922B6115C6
:1046F000710551F08830910538F421912093F10033
:10470000615071090196F3CF21E0089709F020E08C
:104710008091E8008E778093E800CECF2111CFCF33
:104720000AC08091C802882361F0853061F08091D1
:10473000E80083FD0AC08091E80082FFF2CF80E0AC
:10474000089582E0089583E0089581E0089520911E
:10475000CF023091D0022617370748F06115710556
:1047600039F42091E8002E772093E80001C0B901C8
:10477000FC0120E06115710591F18091C802882348
:1047800009F440C0853009F43FC08091E80083FD02
:104790003DC08091E80082FD2FC08091E80080FF3D
:1047A000E9CF2091F3008091F20090E0922B611507
:1047B000710559F08830910540F424912093F1005F
:1047C0003196615071090196F2CF21E0089709F006
:1047D00020E08091E8008E778093E800CBCF211114
:1047E000CCCF0AC08091C802882361F0853061F087
:1047F0008091E80083FD0AC08091E80082FFF2CF3B
:1048000080E0089582E0089583E0089581E00895AE
:10481000982F973068F59093E900981739F07091C8
:10482000EC002091ED005091F00003C0242F762F72
:1048300050E021FD02C09F5FECCF3091EB003E7F46
:104840003093EB003091ED003D7F3093ED003091DF
:10485000EB0031603093EB007093EC002093ED009F
:104860005093F0002091EE0027FDE5CF80E0089501
:104870008F708093E90081E008958091C90287FFDD
:1048800011C08091E80082FD05C08091C8028111AD
:10489000F8CF11C08091E8008B770BC08091C802DF
:1048A000882349F08091E80080FFF8CF8091E800EC
:1048B0008E778093E80008952091E4003091E50020
:1048C00095E64091EC00842F817040FF23C08091D9
:1048D000E80080FD1DC08091C802882399F08530D2
:1048E00099F08091EB0085FD11C04091E40050915A
:1048F000E5002417350729F3915011F09A01E1CF13
:1049000084E0089582E0089583E0089581E00895A9
:1049100080E008954091E80042FFDDCF08950E94B5
:10492000FD240E940525E0EEF0E080818160808317
:10493000E8EDF0E080818F77808319BCA7EDB0E0CF
:104940008C918E7F8C9380818F7E80831092C702A2
:1049500008950F931F93CF93DF930E94FD240E942D
:104960000525C8EDD0E088818F77888388818068AD
:10497000888388818F7D888319BC1092C802109229
:10498000C4021092C6021092C50200EE10E0F801B7
:1049900080818B7F808388818160888342E060E0B2
:1049A00080E00E940824E1EEF0E080818E7F808329
:1049B000E2EEF0E080818160808380818860808386
:1049C000F80180818E7F8083888180618883DF9178
:1049D000CF911F910F910895E8EDF0E080818F7ED7
:1049E0008083E7EDF0E080818160808384E082BF96
:1049F00081E08093C7020C94A924E8EDF0E0808167
:104A00008E7F80831092E20008951092DA00109257
:104A1000E10008951F920F920FB60F9211242F9369
:104A20003F934F935F936F937F938F939F93AF9336
:104A3000BF93EF93FF938091E10082FF0BC08091C1
:104A4000E20082FF07C08091E1008B7F8093E1004C
:104A50000E9480278091DA0080FF1FC08091D800DB
:104A600080FF1BC08091DA008E7F8093DA008091F6
:104A7000D90080FF0DC080E189BD82E189BD09B404
:104A800000FEFDCF81E08093C8020E94522105C044
:104A900019BC1092C8020E9460218091E10080FF41
:104AA00019C08091E20080FF15C08091E2008E7FE6
:104AB0008093E2008091E20080618093E200809127
:104AC000D80080628093D80019BC85E08093C8022A
:104AD0000E9465218091E10084FF30C08091E20056
:104AE00084FF2CC080E189BD82E189BD09B400FE4C
:104AF000FDCF8091D8008F7D8093D8008091E10018
:104B00008F7E8093E1008091E2008F7E8093E200AF
:104B10008091E20081608093E2008091C40288234A
:104B200011F084E007C08091E30087FD02C081E0BE
:104B300001C083E08093C8020E946D218091E10052
:104B400083FF29C08091E20083FF25C08091E100AE
:104B5000877F8093E10082E08093C8021092C402B4
:104B60008091E1008E7F8093E1008091E2008E7F52
:104B70008093E2008091E20080618093E20042E055
:104B800060E080E00E9408248091F00088608093BB
:104B9000F0000E946321FF91EF91BF91AF919F912F
:104BA0008F917F916F915F914F913F912F910F90D6
:104BB0000FBE0F901F9018951F920F920FB60F9275
:104BC00011242F933F934F935F936F937F938F9312
:104BD0009F93AF93BF93CF93DF93EF93FF93C091D6
:104BE000E900CF708091EC00D82FD17080FDD0E823
:104BF0001092E9008091F000877F8093F000789414
:104C00000E9420261092E9008091F0008860809335
:104C1000F000CD2BCF70C093E900FF91EF91DF91B1
:104C2000CF91BF91AF919F918F917F916F915F9144
:104C30004F913F912F910F900FBE0F901F9018959D
:104C40001F93CF93DF93CDB7DEB7AA970FB6F89433
:104C5000DEBF0FBECDBFE9ECF2E08091F1008193A1
:104C600022E0E13DF207C9F70E948B218091E80024
:104C700083FF2EC18091C9029091CA02492F50E052
:104C80004A30510508F024C1FA01EE59FF4F0C9447
:104C9000F427803821F0823809F01AC108C08091C9
:104CA000C5029091C602992389F082600FC080915D
:104CB000CD028F70873008F00BC18093E90080919E
:104CC000EB0085FB882780F91092E9009091E800BD
:104CD000977F9093E8008093F1001092F100D1C08B
:104CE000282F2D7F09F0F4C0882319F0823061F05D
:104CF000EFC08091CB02813009F0EAC0933009F017
:104D000080E08093C6022EC08091CB0281112AC020
:104D10008091CD028F702FEF280F263008F0D8C079
:104D20008093E9002091EB0020FF1CC0933021F418
:104D30008091EB00806214C09091EB0090619093A1
:104D4000EB0021E030E0A90102C0440F551F8A9515
:104D5000E2F74093EA001092EA008091EB0088604D
:104D60008093EB001092E9008091E800877F8093A8
:104D7000E8000E943D24ACC08111AAC01091CB0272
:104D80001F778091E3008078812B8093E3008091EE
:104D9000E800877F8093E8000E943D248091E8002E
:104DA00080FFFCCF8091E30080688093E3001111C5
:104DB00002C082E001C083E08093C80289C08058AD
:104DC000823008F085C08091CB029091CC028C3D5E
:104DD00053E0950779F583E08A838AE289834FB7A8
:104DE000F894DE01139620E03EE051E2E32FF0E07C
:104DF00050935700E49120FF03C0E295EF703F5FAE
:104E0000EF708E2F90E0EA3010F0C79601C0C09688
:104E10008D939D932F5F243149F74FBF8091E80018
:104E2000877F8093E8006AE270E0CE0101960E94DD
:104E3000492316C06091CD027091CE02AE014F5F42
:104E40005F4F0E948D22BC01892B09F441C09091D3
:104E5000E800977F9093E80089819A810E94A723B8
:104E60008091E8008B778093E80032C0803881F52C
:104E70008091E800877F8093E8008091C40280934E
:104E8000F1008091E8008E7772CF811121C080916E
:104E9000CB029091CC0299270297D4F48091E8003C
:104EA000877F8093E8008091CB028093C4020E94A8
:104EB0003D248091C402811106C08091E30087FDEA
:104EC00002C081E001C084E08093C8020E94772183
:104ED0008091E80083FF0AC08091E800877F80937B
:104EE000E8008091EB0080628093EB00AA960FB6F9
:104EF000F894DEBF0FBECDBFDF91CF911F91089513
:104F00000895CF938091C8028823A1F0C091E90051
:104F1000CF709091EC00892F817090FD80E8C82BB4
:104F20001092E9008091E80083FD0E942026CF7056
:104F3000C093E900CF91089587FB082E062687FDD0
:104F4000819567FD61950E942B280EF4919507FCD1
:104F500081950895AA1BBB1B51E107C0AA1FBB1F67
:104F6000A617B70710F0A61BB70B881F991F5A95F5
:104F7000A9F780959095BC01CD01089597FB072E68
:104F800016F4009407D077FD09D00E94AA2707FCE9
:104F900005D03EF4909581959F4F08957095619549
:104FA0007F4F0895A1E21A2EAA1BBB1BFD010DC065
:104FB000AA1FBB1FEE1FFF1FA217B307E407F507C9
:104FC00020F0A21BB30BE40BF50B661F771F881FA5
:104FD000991F1A9469F760957095809590959B013B
:104FE000AC01BD01CF010895EE0FFF1F0590F491B4
:104FF000E02D09940E940228332312F48A1B9B0B94
:105000000C941328A29FB001B39FC001A39F700D01
:10501000811D1124911DB29F700D811D1124911DC0
:1050200008950E940228B7FF0895821B930B0895EC
:105030000E940228A59F900DB49F900DA49F800D03
:10504000911D11240895B7FF0C9418280E94182868
:10505000821B930B0895991B79E004C0991F961742
:1050600008F0961B881F7A95C9F780950895FC0172
:105070004150504030F001900616D1F73197CF01E2
:105080000895882799270895FB01DC0104C08D91BC
:105090000190801921F441505040C8F7881B990BAA
:1050A0000895F999FECF92BD81BDF89A992780B5F0
:1050B0000895A6E1B0E044E050E00C948B28A8E10C
:1050C000B0E042E050E00C948B28262FF999FECFF7
:1050D00092BD81BDF89A019700B4021639F01FBA4B
:1050E00020BD0FB6F894FA9AF99A0FBE0895039668
:1050F000272F0E9466280E946528252F0E94662877
:10510000242F0C9466280196272F0E9466280C9461
:105110006528DC01CB01FC01F999FECF06C0F2BD88
:10512000E1BDF89A319600B40D9241505040B8F765
:065130000895F894FFCF82
:10513600C8003002280850011E0A140101010200AD
:105146000D000D0D01191A1B1C1D1E1F202122D03A
:1051560020F320D4204E214A21D32001E200E90089
:10516600EA00B500B600B700CD008301CC008A0185
:10517600920194012102230224022502260227021B
:105186002A02B300B4006F007000818283E200E956
:1051960000EA00B500B600B700CD008301CC008A56
:1051A60001920194012102230224022502260227EC
:1051B600022A02B300B4006F007000818283F1F40A
:1051C600F5F6F766333790939291F06736950001BE
:1051D600020202020606060909090909090F0F0F4C
:1051E6000F0F0F1515151819191919191919191954
:0451F6001923240055
:00000001FF
